:020000040800F2
:100000000002002071040008C5040008D50400089F
:10001000E5040008F50400080505000800000000DC
:100020000000000000000000000000000D040008B7
:100030001505000800000000F10300080B0200088D
:100040000B0200080B0200080B0200080B0200085C
:100050000B0200080B02000805100008051000083C
:100060000510000805100008051000080B02000824
:100070000B0200080B020008210F00080B02000809
:100080000B020008F50E00080B0200080B02000826
:100090000B0200080B0200080B0200080510000804
:1000A0000B0200080B0200080B0200080B020008FC
:1000B0000D1200080B0200080B0200080B020008DA
:1000C0000B0200080B0200080B0200080B020008DC
:1000D0000B0200080B020008E90E0008150F0008CB
:1000E000051000080B0200080B0200080B020008B4
:1000F0000B0200080B0200080B0200080B020008AC
:100100000B0200080B020008131200080B02000883
:100110000B0200080B0200080B0200080B0200088B
:100120000B0200080B0200080B0200080B0200087B
:100130000B0200080B0200080B0200080B0200086B
:100140000B0200080B0200080B0200080B0200085B
:100150000B0200080B0200080B0200080B0200084B
:100160000B0200080B0200080B0200080B0200083B
:100170000B0200080B0200080B0200080B0200082B
:100180000B0200080B02000800F0D4B97047000011
:1001900070B50C46064600F059F9094B094A1D682E
:1001A0002C44944202D8084A944207D20C2333606C
:1001B0004FF0FF3500F052F9284670BD1C60F9E79A
:1001C00000020020000002203413002019461046CF
:1001D00000F0BCB91946104600F0C0B91323036003
:1001E0004FF0FF307047132303604FF0FF3070472C
:1001F000132303604FF0FF30704702294FF00003D4
:1002000003608CBF00200120704700F08BB9000014
:10021000114B70B500241C60104B114D18682E68EE
:1002200000F09CF80F4B53F820301B68A3F1080234
:1002300096420FD026B13179092904BF0A213171C4
:10024000092103F8041C33F9021C074B2A601980AA
:10025000012070BD204670BD980200208C02002055
:1002600094020020A002002090020020082930B54E
:1002700003791AD9082B14D842791A4B53F8225013
:1002800000F108047DB12D68856053F822502C6080
:1002900043F82240144A44790123A34014682343BD
:1002A0001360017130BD8460F2E7082BF9D94579FC
:1002B0000C4B53F825203AB11468A2420BBF002220
:1002C000246843F825201460427953F82230002B2B
:1002D000E7D1054C012303FA02F2236823EA020363
:1002E0002360DEE7A00200208C02002008B50A4B44
:1002F0001B681A79082A02D95B7983420AD900F06F
:10030000B0F818B1054B01221A6008BDBDE80840DD
:1003100000F066B808BD00BF9402002098020020DB
:1003200008B500F093F8094B094A1B88094D1BB228
:10033000002442F82340084A286813682146013BFC
:100340001360FFF793FF2C6000F046F89002002046
:10035000E0020020940200209C0200200023C2073B
:1003600001D51846704740080133F8E7134423F0DD
:10037000030310B54FF077321C1F43F8042C6207BB
:1003800042BF4FF0883243F8082CA3F108044FF025
:10039000807304E909000F4B44F80C3C002344F837
:1003A000103C032344F8143C2246022344F8183C32
:1003B000012344F81C3C42F8201D0B2342F8043D65
:1003C000013B032BFAD120466FF0020340F8443D75
:1003D00010BD00BF2103000800F03CF801DFFEE77C
:1003E000024A536843F080535360704700ED00E0C9
:1003F000EFF3098020E9F00F40F804ED02490968A5
:10040000086000F003F8000094020020FFF700FFEE
:1004100004480068016801C9B1E8F00F81F3098858
:100420000047000094020020BFF34F8F0549064BA0
:10043000CA6802F4E0621343CB60BFF34F8F00BF82
:10044000FDE700BF00ED00E00400FA05EFF31080C7
:1004500072B6704762B6EFF31080704780F3108871
:100460007047EFF30580C0B27047704770470000D7
:1004700008B5FFF7FAFF0E4A0E4B0F498B420ED319
:100480000E4B0F4A002193420ED3FFF7EFFF00F00F
:100490000DFA03F0BBFEBDE8084000F053BA52F875
:1004A000040F43F8040BE9E743F8041BEBE700BF34
:1004B0006C530008000200208C0200208C020020F7
:1004C0003413002008B50249042000F00DFA00BFE3
:1004D0005C51000808B50249052000F005FA00BF8C
:1004E0003651000808B50249062000F0FDF900BFAA
:1004F0004951000808B50249072000F0F5F900BF8E
:100500000451000808B50249082000F0EDF900BFC9
:100510006851000808B50249092000F0E5F900BF5C
:100520001651000808B502490A2000F0DDF900BFA5
:1005300028510008034B044A4FF4E131002000F039
:100540000DBC00BF04020020290C00080A46014629
:10055000014800F074BB00BF0402002010B50A4639
:100560000C460146002000F0A3FB204610BD0020F1
:1005700000F0EEBD034B1968024611B9084600F0C1
:10058000C7BD7047A403002010B5094A136843B1E2
:100590009C6881688C4207D303D15C6841688C42B7
:1005A00002D90360106010BD1A461B68EFE700BF58
:1005B000AC030020F0B51F4E1F4D33681F4C0133B4
:1005C00033601F4B00201A6818602B6822601946A0
:1005D0000746B64621B1DEF800C08E68664503D9ED
:1005E00000B1296027B9F0BD0F4601200968F1E785
:1005F00000213960DAB163B151685868814294BF13
:1006000011461946084612681B6822B9036021602A
:10061000F0BD1146F6E70BB90260F8E755685E6871
:10062000B54294BF15461D4605602846EBE723609A
:10063000F0BD00BFA8030020AC030020B4030020DD
:10064000B00300202DE9F0412C4F2D4C01233B60DD
:10065000236893B9FFF7AEFFFFF789FF0130FBD0A6
:1006600000254FF0000823685BB9FFF780FF854243
:1006700024D9FFF79FFF0025F5E7FFF778FF054630
:10068000EFE75E68FFF773FF854204D8864202D920
:10069000361A132EE9D823685E68FFF768FF854293
:1006A00001D88642F7D823681A682260C3F804800C
:1006B000C3F80880DA6818699047D4E723686BB1FB
:1006C0005E68FFF754FF063E14308642CBD300230A
:1006D0003B603046BDE8F041FFF74CBFFFF747FFF6
:1006E00085420646C5D810F1140F04D3FFF73FFF2B
:1006F0008642FBD9BDE74FF0FF36E8E7A4030020B0
:10070000B4030020144B1A6882420FD112681A6099
:100710001AB150680638FFF72DBF4FF0FF30FAE7E7
:10072000904202D102681A60704713461A68002A84
:10073000F6D10A4A13681BB9094A13683BB97047D6
:10074000984202D10368136070471A46F2E7984254
:10075000F8D01A46F1E700BFB4030020B003002030
:10076000AC03002008B500231846054A054900F0EF
:1007700015FD4FF0FF30BDE80840FFF7FBBE00BF9E
:100780004506000840420F00F8B504460D46FFF745
:10079000EEFE002385420646236011D3A5F10A032D
:1007A00083420DD20A35FFF7E2FE8542FBD3FFF705
:1007B000DEFE8542FBD8E368206998470020F8BD3B
:1007C000FFF744FE63680746002B33D1A368002B74
:1007D00030D11A4B65601A681B68B54238BF0132C8
:1007E000A260A2689A4206D92046FFF7CDFE38469D
:1007F000FFF734FEE2E7B5420FD9114B19461A68EC
:1008000012B15068854213D222601C600B689C4272
:10081000EDD1A81FFFF7AEFEE9E70A4A136813B14E
:1008200059688D4202D223601460E0E71A46F5E76A
:100830001346E4E72046FFF765FFCAE7A803002058
:10084000B4030020B003002038B50446FFF7FEFDD6
:100850006368054633B9A36823B92846BDE8384024
:10086000FFF7FCBD2046FFF74DFFF6E7C36870B504
:1008700004460D46C3B1FFF7E7FF092D0CD8FFF77B
:1008800076FE0646FFF773FE801B8542FAD8E368C2
:100890002069BDE870401847FFF769FE2918204617
:1008A000BDE87040FFF770BF70BD000008B50121C2
:1008B000094800F045FB0121084800F041FB0121F7
:1008C000074800F03DFB0121064800F039FBBDE878
:1008D000084000F0F3B800BF0D0C02400C0C0240C1
:1008E0000E0C02400F0C024008B5084B1A683AB9CA
:1008F000012207481A6003F0CFFC064803F0CCFC45
:10090000FFF7A4FD00F0D8F8FFF78EFDB803002034
:100910007C5100089851000808B500F0DDFC034840
:1009200003F0BAFC00F0A0FC002008BDAB510008A9
:1009300008B5034C2368012000F040F9FAE700BF36
:10094000BC0400201FB5FFF781FD0E4B0E481B684D
:10095000029300240D4B00930F220C234FF480715F
:10096000019400F045F80A4B0A481B6802930A4BB1
:10097000009307220C234FF4C061019400F038F873
:10098000FFF72AFD18020020BC03002031090008EF
:100990001C020020C00400201909000808B5FFF758
:1009A00055FD094B1B681A79082A07D95A79074B54
:1009B00053F8221011B1096843F82210FFF74EFDD9
:1009C000BDE80840FFF70CBD94020020A002002003
:1009D00030B54C7901F10802036813B98B600260ED
:1009E00030BD13F8035CAC42F8D31846F4E70000BE
:1009F0000F2A2DE9F84F07469046994627D810F060
:100A000003031CBFC3F10403C91AA1F1240118BFD9
:100A1000FF1821F00306FFF719FD254ABC1983468C
:100A2000012352F823500FFA83FA9DB10133212B91
:100A3000F7D15846FFF712FD6FF08A0A35E0012121
:100A40002046FFF713FC5846FFF708FD2DE06FF036
:100A5000150A2AE042F823400B99A4F806A0334671
:100A60003A460A98FFF782FC124A20604FF0FF33A3
:100A7000E361136884F80580013319F0010F2571D3
:100A8000A560E56025616561A56125621360D6D129
:100A90000A212046FFF7EAFB19F0040FD3D158468C
:100AA000FFF7DCFC4046FFF721FC5046BDE8F88F1D
:100AB000E00200209C0200207047000010B53C4C72
:100AC00000F06CFC0022A260236823F0867323F4FC
:100AD00080332360E260236843F48033236023681B
:100AE0009803FCD54FF08051002000F0BFFA314A46
:100AF000136843F400431360A36823F0F003A3607A
:100B0000A368A360A36823F46043A360A36843F4CD
:100B10000043A360A36823F4E053A360A36843F4F5
:100B2000A053A36000236360636843F480036360A1
:100B3000636843F008036360636843F4A843636039
:100B400063686360636843F0E0636360236843F055
:100B50008073236002F5E43213689901FCD5164BCB
:100B600000211960196841F400711960196841F495
:100B700080611960196821F00F011960196841F04E
:100B800005011960936823F003039360936843F0B1
:100B900002039360064B19469A681207FCD51A683F
:100BA00022F001021A600B689B07FCD410BD00BF45
:100BB0000038024000700040003C0240174B93F99F
:100BC0000010042806D8DFE800F00307101C1C0002
:100BD00000221A700846704701221A70104A1369E1
:100BE00023F00403136130BFF4E702221A700D4AA8
:100BF000136823F003031360094A136943F00403E5
:100C0000F0E703221A70074B1A6842F00E021A60CE
:100C10005A6842F480725A60EEE700BF200200205A
:100C200000ED00E00070004038B50446043000F0EC
:100C300008FB0546204600F08BFB284638BDF8B57A
:100C400004460E461746051D3A463146284600F032
:100C5000E3FA00B1F8BD0121204600F049FBF3E7BB
:100C60004209012300F01F0003FA00F0014B43F892
:100C70002200704700E100E0024B1B680BB1FFF758
:100C80008DBE70479802002008B50B689B0608D5FA
:100C9000064B496803EBC002C9B253F830305068C4
:100CA0009847BDE80840FFF7E7BF00BFD00A002023
:100CB0002DE9F84306460C461546FFF7D2FBDFF850
:100CC000849078B118235E43254459F80630AC422D
:100CD00001D1BDE8F8831A681206FCD514F8012B7F
:100CE0005A60F4E7134F4FEA86084744012138461B
:100CF00000F0FEFA182303FB06960F48F17C0F4A1A
:100D00000729D8BF024601F00701102013FB010399
:100D1000D118ADB2CC604D60D158094841F0010105
:100D2000D1504044012100F0E3FA3846BDE8F843D1
:100D300000F00EBBC80A00200060024000640240C0
:100D4000C00A0020F8510008034A182303FB0020C2
:100D50004168407C00F08AB9F851000801282DE96B
:100D6000F84F05460C4600F2A78018214143544F26
:100D700007EB01087E58534941F8302001EBC001D0
:100D80004FF000094B60504B43F820904F48012131
:100D900040F8259000EB850000F0AAFAD8F808B0DA
:100DA0004946584600F0CCF8D8F80C900121484646
:100DB00000F0C6F898F810A05846514600F0FAF82E
:100DC0005146484600F0F6F82846FFF7BDFF98F870
:100DD00011302401002B4FD13D48B0FBF4F003F05B
:100DE0004DF8804603F0F2F984B2204603F04AF849
:100DF0000146404602F090FF4FF0834103F096F821
:100E000003F0E4F9240100F00F00A4B204438023AE
:100E1000B46073610023336142F20C03F360182362
:100E200003FB0573DC7C072C28DC4FF40011022047
:100E300000F01CF9274A1820102104F0070310FBCA
:100E4000031300FB05702449057D90F9120002EBA5
:100E5000030E41EA4561D150331DCEF8083000231E
:100E6000CEF81430FFF7FCFE062C0EDC04F10B006C
:100E700040B2FFF7F5FE0EE01848AEE74FF48001F0
:100E8000022000F0F3F8164AD5E7072C0AD1154BDB
:100E90004FF400425A60F36843F02003F3600020EF
:100EA000BDE8F88F0C2C02DC04F13000E0E70F2CD9
:100EB000F1DC04F13700DBE74FF0FF30BDE8F88FDD
:100EC000F8510008D00A0020C80A0020C00A0020FB
:100ED00080DE8002006002405004010000BD010578
:100EE0000064024000E100E001490020FFF7CCBEB1
:100EF0000044004008B5054B05484FF40012DA6085
:100F000000F026FABDE80840FFF7B6BE00600240D8
:100F1000C00A002001490120FFF7B6BE004800408A
:100F200008B5054B05484FF000629A6000F010FAD2
:100F3000BDE80840FFF7A0BE00600240C40A0020E0
:100F4000F8B50D460126C0F3832120F00F0400F010
:100F50000F0706FA01F1022000F088F807FA06FEF2
:100F60000323226803FA0EF3D8430240226022686A
:100F700005F0030101FA0EF111432160E26810400F
:100F8000E060E168C5F3810202FA0EF20A43E26012
:100F90006268BE4022EA060262606268C5F300151C
:100FA000BD4015436560A268B6B21343A36000203C
:100FB0006683F8BD20F00F03F0B500F00F041D6844
:100FC00067000326BE4025EA06051D601D68022253
:100FD000072C02FA07F242EA050294BF002401241A
:100FE0001A6003EB840300F007001A6A80000F24E4
:100FF000844022EA04021A621A6A01FA00F01043DD
:101000001862F0BD2DE9F0410F4D104F6E692A684E
:10101000002416404FF0010808FA04F31E4206D0DF
:101020006B6107EBC40357F83420586890470134CC
:10103000102CF1D1064B1B681BB1BDE8F041FFF746
:10104000ADBCBDE8F08100BF003C0140E00A0020DB
:1010500098020020034B044A00280CBF1046184693
:10106000704700BF00BD010580DE8002042808D85B
:10107000DFE800F0030A0F1419000D4A136C19433E
:101080001164BFF34F8F7047094B5A6C1143596479
:10109000F7E7074B1A6B11431963F2E7044B5A6BDE
:1010A00011435963EDE7024B9A6B11439963E8E7EB
:1010B000003802402DE9F843124ADFF8508003015E
:1010C0000746D5582E69EB6800241E4008EBC0097E
:1010D0000223A3401E4209D0EA68D9F8040022EA9C
:1010E0000303EB60214658F8373098470134042C4D
:1010F000EED1054B1B681BB1BDE8F843FFF74EBCB2
:10110000BDE8F8832852000898020020600B0020F8
:10111000032910B516D80D4B00011C181858636828
:101120001A4001F10C0300EB83035A6002690223A9
:1011300003FA01F122EA01020261C3681943C160A6
:10114000002010BD4FF0FF3010BD00BF2852000836
:101150000001024B1B58586A704700BF2852000814
:10116000034B00011A58136843F0010313607047E2
:1011700028520008074B03EB00100121437B5AB2B1
:1011800003F01F0301FA03F35209034941F8223027
:10119000704700BF2852000800E100E001282DE957
:1011A000F84305460F4629D8164E1749040106EBA9
:1011B000040841F8302098F80C9001EBC001484633
:1011C0004B60D8F80810FFF751FF3659D8F80430B3
:1011D0000024346048467460F362FFF73BFF01234C
:1011E000B0FBF7F00138B06273612846FFF7C2FF29
:1011F0002846FFF7B5FF2046BDE8F8834FF0FF30E3
:10120000BDE8F88328520008600B00200020FFF79B
:1012100051BF0120FFF74EBF70B514461CB1856861
:10122000C3689D4201D1101B70BD86680568731CA0
:1012300083604368013B3340013CEB5C01F8013BB8
:10124000ECE7C268436830B58468121B9A4208D044
:10125000C2680468013B1340551CC560E15400207E
:1012600030BD4FF0FF3030BDF0B518488DB003F001
:1012700087F801A801F098FD28B3BDF90400144EC9
:10128000144F00F071FC044600F1E00508223146DD
:10129000204602F0DFFF38B12378FF2B10D16378AE
:1012A00003F00F03022B0BD1237CDB0708D421466C
:1012B000282202A802F060F802A9384602F0ECFFEA
:1012C0003834AC42E2D100200DB0F0BD48520008E5
:1012D000965200086F52000808B5FFF743FA01F074
:1012E000B1FE00F021F9BDE8084000F0C7BD0000E4
:1012F00070B504460D46FFF7A9F8236806463BB9CA
:101300004FF0FF332360FFF7A9F80125284670BD91
:10131000C5B10E4B1D6802212846FEF7A7FF2368C2
:1013200001330AD105F1080323600023AB60304686
:10133000FFF794F8FFF754F8E7E729462046FFF750
:1013400047FBF4E7FFF78AF8E0E700BF94020020CC
:1013500070B50446FFF77AF8256806461DB9BDE862
:101360007040FFF77BB86B1C02D100232360F6E7C7
:1013700028460A2150F808392360FEF777FF2368D2
:1013800013B94FF0FF33236015F8034C3046FFF7D5
:1013900065F82046BDE87040FEF7A8BF0F4BD3F8B4
:1013A000882042F4700210B5C3F888204FF0006224
:1013B0009A600B4C102283F822200021DA77601803
:1013C0000131522980F80023F9D11A6942F0100244
:1013D0001A615A6942F400725A6110BD00ED00E0D2
:1013E00000E100E0002101F027BF38B5CBB20021B9
:1013F00014460246084601F0E3FC054620B92046A3
:10140000FFF7F0FF284638BD94F9103001330AD1B8
:10141000A36882681B7903F03F03214620461371BD
:1014200001F03EFF04466C60ECE738B58B680C4673
:101430005880054600F098FB6368002243B9B0F875
:10144000E830934208D22046BDE83840FFF7CABFD3
:10145000D9685B680A44F1E72146284601F071FC2F
:101460000028F0DD38BD00002DE9F0478C68054606
:1014700088461646002362B95BBAA380A379FF2B86
:101480000DD196F91030012B07D0022B2FD03B2322
:1014900004E0D16852680B44EDE72923A371E37996
:1014A00013B935BB4023E37104F1080710221C492E
:1014B000384602F0CFFE824670B904F11809194986
:1014C0001022484602F0C6FE0146C0B91022384636
:1014D00002F0DAFE0123E3754146304601F0E0FCFC
:1014E000002819DA831C08BF0020BDE8F0873A23E2
:1014F000D4E7284600F038FB90F8EA30D3E74946B5
:101500005246284600F0EAFB01460028E4D01022AB
:10151000384602F0AEFEDFE70020BDE8F08700BFEE
:10152000C6520008A65200081FB50A4CB4F9003094
:1015300063B9094A0193094B0292009304220823DC
:101540004FF480610648FFF753FA2080B4F9000099
:1015500004B010BD700F0020815200084D17000824
:10156000700B0020292B2DE9F8438146884614464C
:101570001D4621D03A2B0CBF02230023292D88F8C9
:1015800010301BD03A2D19D00027D8F8043093F929
:101590001060012E14D01FB10121204601F03AFE47
:1015A000234640F201222946012001F09FFB00BBA7
:1015B0002046FFF717FF1CE00123DFE70127E4E7E0
:1015C0002946304601F050FC00B927B101212046E0
:1015D00001F020FE0026234640F20122154998F929
:1015E000100001F083FB10B92046FFF7FBFE002E30
:1015F000D1D0E7B1292D07D03A2D18D12146484640
:10160000BDE8F84302F06CB900232374616819B196
:1016100091F91030012B06D0012323742046BDE838
:10162000F84300F009B8204601F03AFEEEE7BDE8C5
:10163000F88300BF0000FFFF2DE9F0414FF0FF31BC
:10164000074601F03AFCC8B18368B3F902403E4650
:101650003846A8B9BB681B7803F0F003602B1FD194
:10166000384601F0F7FD0546D0B10122282101F0EE
:101670001FFD00232B7438BB284612E00446E6E722
:1016800090F91030012B08D1C368282B05D183684D
:101690001B7803F0F003602B07D006464068D8E7BC
:1016A0003846BDE8F041FFF79DBE3D468768EB68D0
:1016B000B98849BA89B2994208D32A4600239ABB0D
:1016C000283B994205D9D7E72E46EFE7284601F097
:1016D0005BFD07F1180810221A49404602F0BAFDD6
:1016E000D0B108221849404602F0B4FD38B13B7E23
:1016F000FF2B05D17B7E03F00F03022B00D1DCB959
:101700004146002000F08EFA002C08BF0446B0FAD3
:1017100080F040090028AFD1BB792A4631462046E7
:10172000BDE8F041FFF71EBFD068034492F91000F6
:101730000128C5D05268C2E74146204600F054FA5D
:10174000E5E700BFA6520008965200082DE9804840
:10175000A1B002AF0023FB62A3F580333B63864B4D
:10176000DFF81C921B88BB86082107F1380002F0C5
:101770007FF807F12C01012001F054FB40F2052312
:10178000FB8340F2032840F2012407F1140002F029
:101790006BF8FB8AB3F5017F1AD8434580F0C0800F
:1017A000A34228D040F202229342EED1BB691D46EB
:1017B00093F9103001332BD1AB682846B3F902609E
:1017C00001F048FD0446D0B92846FFF70BFEDAE7E2
:1017D00040F21222934200F0AD8040F21722934271
:1017E00000F0AC80B3F5047FCFD1BA69537F23F00A
:1017F00008035377C7E7B869FFF71EFFC3E74368DD
:101800009A46504601F026FD054628B92046DCE7F9
:10181000AA462C460026F4E7A245836818BF6060FC
:101820001A461B7ED0F804A008BF0446FF2B21D126
:101830007EB907F1240001F0B7FA0028E6D00021B4
:1018400022460846B7F92460FFF7CFFD044600287A
:1018500099D0524629463046FFF706FE0028D5DBD0
:10186000A268137943F04003137121463046FFF715
:10187000DCFD88E7134618331022494618467B6082
:1018800002F0E8FC48B17968002E5BD107F1100046
:1018900000F0C8F90646002859D05246294630467D
:1018A000FFF7E2FD0028B1DB29460022CB6849683A
:1018B0001A440029FAD10123084601F0DFFB06464D
:1018C0000028A3D083689A46EA68A968504602F0C7
:1018D000D0FCEB686D6852461A449246002DF3D155
:1018E0002046FFF77FFD254B3146B3F9000001F09C
:1018F00035FA00283FF747AF304666E7524629469B
:10190000FFF7B2FD002832DBF97B224607F1240005
:10191000FFF76BFD014668B33046FFF786FD29E00F
:101920006FF0850307F11C0107F114003B6201F021
:1019300073FF28E7B86900F043FD24E7B86900F0B9
:10194000CFFD20E7304600F04FF90028A5D107F180
:101950007801082301F8693D009432467B6807F15D
:10196000240001F0DFF8EB4606460028C6D12046E9
:10197000FFF738FDDD4606E790020020700F0020DB
:10198000A65200080121FFF7B3BC2DE9F84300F18E
:10199000E005074628468846FFF7F4FF00244FF08D
:1019A000380909FB04764146304601F090FC58B1F5
:1019B00010220021304602F067FC002333742846D1
:1019C000BDE8F843FFF7C4BC0134042CE9D1F6E7C5
:1019D00008B51022034902F03DFCB0FA80F040093E
:1019E00008BD00BFC652000810B5082209490446C8
:1019F00002F030FC48B12378FF2B08D1607800F06A
:101A00000F00831E5842584110BD012010BD002018
:101A100010BD00BF965200082DE9F04F074685B073
:101A20000E4692469846054600F1E00B00243146EA
:101A30002846A94601F04BFCF8B92846FFF7C8FF35
:101A400010B1002C08BF2C463835AB45EFD1A1466C
:101A50009CB110223146204602F00BFC84F811A004
:101A600084F810803378FF2B0BD148F0010884F8FC
:101A7000108040F2112363866463484605B0BDE8D8
:101A8000F08F3046FFF7B0FF18B1237C63F07F037F
:101A90002374B7F8E63003F00303012BE9D040F2DA
:101AA000FF220023CDE900234FF080730293FF2330
:101AB0008DF80C30737B8DF80D30F389ADF80E3056
:101AC0008022002369463846FFF7A6FFD1E7038846
:101AD0005BBA23F03F031B041B0C4FF6C06293421A
:101AE0000AD00378FF2B09D1437803F00F03052BAD
:101AF00014BF0E2005207047052070470E20704748
:101B00002DE9F0470025804691461F460C462E469B
:101B10004FF0010A3FB13A780AFA05F31A421AD097
:101B2000237CDB0717D42046FFF752FF98B94946BC
:101B3000204601F0E1FB37B999F80030FF2B02D0C5
:101B4000637C834207D8B04205D9B8F1000F01D0B9
:101B5000C8F8004006460135042D04F13804D9D1F7
:101B60003046BDE8F0870000034BB3F9E420824221
:101B70000CBF184600207047740F00202DE9F0417B
:101B80000D4617469846FFF7EFFF044618B90024A4
:101B90002046BDE8F0810029F9D00846FFF718FF7C
:101BA0000028F4D1802FF2DC04F1E0063046FFF784
:101BB000E9FE43463A4629462046FFF72DFF0446F4
:101BC0003046FFF7C5FBE3E710B538B90548B0F973
:101BD000E43033B1BDE81040FFF7D7BEFFF7C4FFD4
:101BE000F8E710BD740F0020F8B50F46FFF7BCFFF3
:101BF000044668B100F1E0052846FFF7C3FE394608
:101C0000204601F064FB064620B12846FFF7A0FB02
:101C10002046F8BD3834AC42F1D12046FFF798FB9E
:101C20003446F5E738B5084C0546B4F9E40025B963
:101C3000FFF7DAFF28B9002038BDFFF7D5FF28608D
:101C4000F8E7B4F9E40038BD740F00202DE9F34142
:101C500002AD00260E4C45F8046D8846074604F197
:101C6000E000FFF78FFE3346424621462846FFF745
:101C700047FF50B1019BB4F9E4403B600548FFF7D2
:101C800067FB204602B0BDE8F0810446F6E700BFDE
:101C9000740F0020541000202DE9F34102AC0027FE
:101CA000884644F8047DFFF75FFF00F1E005064633
:101CB0002846FFF767FE20463B4642463146FFF77F
:101CC0001FFF044628462CB1FFF742FB019802B0E3
:101CD000BDE8F081FFF73CFB2046F8E72DE9F04F27
:101CE00087B00F461546FFF73FFF00F1E00380463F
:101CF00018460193FFF746FE0122002103A802F0D7
:101D0000C3FA4FF0FF334646C246009300244FF01B
:101D100001099AF80020FF2A0ED05046FFF758FE1E
:101D200050B9002D40F085809DF80C10009409FA00
:101D300004F20A438DF80C200134042C0AF1380A0D
:101D4000E7D1009B013300F0958004AD22460021CD
:101D5000284602F099FA3B78FF2B71D197F8019051
:101D600009F00F094FF0000A54469DF80C100123AA
:101D700003FA04F2114224D039463046B34601F04A
:101D8000A6FA002847D13046FFF72EFE002863D17F
:101D90003046FFF79CFE814560D12A5D0432D2B205
:101DA0002A55524588BF4FF0040AB2694AB12A5DEC
:101DB0000132D2B2524513462A5538BF53465FFA14
:101DC00083FA0134042C06F13806CED10122002119
:101DD00003A802F059FA00209DF80C2001460124C6
:101DE0006E5C564504BF04FA01F0024301F10101A3
:101DF00004BFD2B201200429F2D108B18DF80C2021
:101E000006A8002340F8043D3A4603AB4146FFF7DD
:101E100077FEDDF814B0BBF1000F03D1009B382230
:101E200002FB038B0198FFF793FA584607B0BDE811
:101E3000F08F5046FFF7D8FD00287FF475AF7BE7A1
:101E40003846FFF7D1FD20B93846FFF740FE8146FE
:101E500088E74FF0020985E702209CE7A5D92A5DB3
:101E60000232D2B25245134638BF53462A555FFA62
:101E700083FA9AE74FF0000BD4E700002DE9F04712
:101E80008AB003AE304600F08FFFDFF8B8A080467E
:101E900000244FF00809444502D10AB0BDE8F0879C
:101EA00036F91400FFF760FE0546002847D000F120
:101EB000E0073846FFF766FD36F91400CDF80090CC
:101EC00004AB0022072100F056FF00280FDB082298
:101ED00004A908A802F0CDF90822514606A802F08C
:101EE000C8F90023402206A92846FFF795FD0223E2
:101EF00036F91400009300220DF10E03092100F0C1
:101F00003AFF002806DBBDF80E30B3F5A06F28BFFE
:101F1000A5F8E830002336F9140000931A46192179
:101F200000F029FFB5F8E6300028CCBF43F080036D
:101F300023F08003A5F8E6303846FFF709FA0134AC
:101F4000A9E700BF9652000813F1860F2DE9F3416F
:101F50000746884616461C460BD001F053FE054640
:101F600050B9032300933246A3B24146384601F0EC
:101F7000F5FD02B0BDE8F081027FA3B29A4200F104
:101F800014070CD031462C772246384602F071F9FE
:101F90000321284602B0BDE8F04100F061BC2246B2
:101FA0003946304602F056F90028EBD1E1E700004F
:101FB0002DE9F04F1D46D3798BB0FF2B804603915E
:101FC0001646149C15D16B789BB9172C11D92B7A16
:101FD000FF2B0ED002F1080926491022484602F0D4
:101FE00039F948B105F108014046FFF7FDFD824689
:101FF00058B90BB0BDE8F08F0D221F4906F118004B
:1020000002F028F90028F4D0ECE70023183C1F4622
:10201000002C16DC04AA49464046FFF795FF4946C6
:10202000102206A802F025F9337E00220092A3F1C7
:10203000FF0253425341514606AA404600F046FB78
:10204000D7E707F1180205EB020BAA5C012A09D1B8
:1020500004AB00932A7803985B46314600F060FC9D
:10206000031EC6DB9BF8012007EBC207BFB2A4EB3F
:10207000C204CDE7C6520008B65200082DE9F04F61
:10208000924687B0894603F108011D468046109E9E
:1020900001F0B8FD9AF80730FF2B044640F0BA80F3
:1020A0006B78002B40F0B680172E40F2B3802A7A6E
:1020B000FF2A00F0AF80002800F0AC80183E1F46D9
:1020C000002E44DC4FF0FF314846039300F0F5FE4C
:1020D000039B00B18068627F02F00702022A52D19E
:1020E00028B102781AB14278002A40F09A8004A9F7
:1020F0001A462377A4F81E8004F1140002F0B9F800
:102100002B7959064CBF07210321204600F0A8FB7C
:1021100095F90430002B637F32DA43F00803002680
:10212000444F6377B0462568002D73D02B68236039
:1021300069682E60B7F9000000F003FE002803DC98
:102140000021686801F078F8C5F80480EBE707F132
:10215000180205EB020BAA5C022A09D104AB2A780B
:10216000009351465B46484600F016FC031E51DBC7
:102170009BF8012007EBC207BFB2A6EBC2069FE7A0
:1021800023F00803CBE700284FD00278002A4CD078
:102190004278002A49D0002B49D0227F934246D072
:1021A0001A4604A904F11400039302F053F8B0FA9C
:1021B00080F67609039B03E0267F003618BF0126D0
:1021C0002A7992060BD456B19BB1637F03F00703C3
:1021D000072B1FD10321204600F042FB1AE043B138
:1021E000A4F81E8023771A4604A904F1140002F013
:1021F00040F82B795B0610D50721204600F030FB14
:1022000095F90430002B637FB4BF43F0080323F03B
:102210000803637707B0BDE8F08F002EF0D00321EC
:10222000EBE7002B7FF463AFF4E7002BC4D000266C
:10223000C6E700BF700F00202DE9F04F87B0904631
:1022400003911C460646109FFFF78EFC08F1080913
:10225000054608225649484601F0FCFF0290C8B9DD
:1022600098F80830FF2B15D098F80730FF2B11D1C4
:1022700063787BB90F2F0DD94946304601F0C2FC77
:1022800058B90B230093024603464946304601F0F5
:1022900065FC58B907B0BDE8F08F437F1A0757D5E2
:1022A000E288002A54D123F008034377E1888BB2F7
:1022B0006BB1404BDFF804E11B8849BA89B200F1E9
:1022C00034021BB20EFB01F1203001F035F9237905
:1022D0000BB185F8EA306279374B03EA0223B5F88F
:1022E000E620C2F30D021343A5F8E630A068A8B1BA
:1022F000D5F8EC3090FA80FA53450FD001F00CF984
:102300000A22B0FBF2F303FB12000530C5F8ECA083
:102310000AFB00FABAFBF2F2C5F8F020E36813B149
:102320001BBAC5F8F43005F1E000FFF711F8A7F18A
:10233000100B0027BBF1000F0DDC3046029B04AAF6
:102340004946FFF701FE05F1F800FEF77DFAA1E727
:1023500043F00803A9E707F1100304EB030AE35C69
:10236000032B1ED0052B14D0012B0AD104AB0093F4
:10237000227803985346414600F0D2FA031E029396
:1023800088DB9AF8013007EBC307BFB2ABEBC30B96
:10239000D0E752462178304600F030FB0028F0D1DB
:1023A00078E752462178304600F044FBF6E700BF5C
:1023B000965200089002002000C0FFFF40420F002C
:1023C0002DE9F041437F03F00703022B86B004465A
:1023D00001D0052B38D194F87420B4F91E50012A8D
:1023E00075D9022B33D14FF0807340F2FF200021CA
:1023F0000493FF238DF81430CDE90201637C8DF83E
:102400001530638AADF81630013A84F87420A5BB04
:1024100001AE304600F0C8FC04F104080746BD4296
:1024200022D12D4B04F13C05B3F900602846FEF79C
:102430000BFA40F21223A4F8523004F15002334652
:102440002649284601F078F806B0BDE8F081211D44
:1024500003C902AB83E8030004F10C0393E8030013
:1024600006AB03E90300CFE736F9150002AB42469D
:10247000002100F0B7F90135D1E72846FFF774FBDA
:102480000646221D02AB06F1E005B4F91E0000214C
:1024900000F0A8F901212846FEF72AFF0E4BD6F8D6
:1024A000F470B3F9008004F13C063046FEF7CCF935
:1024B00040F21223A4F852303046434604F1500251
:1024C000394601F039F82846FEF742FFBCE7211DE6
:1024D000284601F0B5FBB7E7700F002040420F001F
:1024E000437F03F00703042B04D0072B04D10321FF
:1024F00000F0B6B90521FBE7704710B50446084661
:102500002378FF2B14D018230022872101F03FFAF3
:1025100078B1836800221A715A719A71DA71216850
:102520006268DA609960A168E2685A61196110BD59
:10253000002010BD38B50B78FF2B05460C46104621
:1025400016D018230022882101F021FA88B183686F
:10255000002225F01F051D71DA719A715A712168E8
:102560006268DA609960A168E2685A61196138BDF1
:10257000002038BD10B5002304461046CA1D02F0E5
:10258000F802194600F07AFD20B182681470C36821
:10259000DB08537010BDF8B516460F461A46B11C3D
:1025A000FFF7E8FF044660B18568C2680235023A69
:1025B0000021284601F068FE32463946284601F0DF
:1025C00058FE2046F8BD13460A4601460120FFF793
:1025D000E2BF13460A4601460220FFF7DCBF70B592
:1025E00006460846194601F05DFA044678B183684C
:1025F000FF22DA7100231A461946184600F0E0FB64
:10260000054630B92146204600F04AFE2C462046B9
:1026100070BD83685E804460F8E7002100F00CBE66
:1026200030B585B0022300930D460DF10E03002254
:102630000521044600F09FFB002803DBBDF80E30A7
:10264000062B13D80823009300222B460221204694
:1026500000F091FB002805DBADF80E00BDF80E0080
:1026600005B030BD0023ADF80E30F7E70823009326
:1026700000222B460321204600F07DFB0628E1DDE9
:10268000EAE7000038B5002001F0FCFA044660B922
:102690000D4D286801F0F6FA034618B901F0F2FA78
:1026A000034678B12B60181D38BD637F03F0070324
:1026B000013B012B04D9044B00221A60201D38BDB8
:1026C0002046E1E7204638BD881000202DE9F74379
:1026D0000A9C8846994607461646FFF745FAB0F821
:1026E000E63099071DD4002510223A49304601F002
:1026F000B1FDF8B910223849304601F0BAFD022385
:102700007370B9F1000F19D069463846FFF788FF9A
:10271000A0B1C1B222466846FFF75BFF68B9204608
:1027200024E03846FFF720FAB0F8E6305A07DAD549
:102730008025D9E745F04005E3E704462CB198F839
:102740001030DB0758BF45F0200528462246414699
:10275000FFF7F0FE05460028E1D00146002332468F
:102760003846FFF73CFF044618B92846FFF755FFE7
:1027700024E098F81030DFF8688013F0010F20D0C3
:1027800000F0CAFE31468146384601F03BFA00F1BE
:10279000580605463046FEF757F810492C6740F2B8
:1027A0000223B9FBF1F0A5F86E3001FB1091B8F9E6
:1027B000003005F16C02304600F0BEFE03B0BDE80B
:1027C000F0830146B8F9000000F0BBFA0028F5DC00
:1027D000A5E700BFC65200088652000840420F001D
:1027E000700F00202DE9F3410746164698460D4626
:1027F00029B90A463146FFF771FA054670B16946B4
:102800003846FFF70DFF90B1C1B200226846FFF7CE
:10281000DAFE044618B9FFF700FF1CE00446304614
:102820002146FFF76AFE064618B92046F3E704463C
:10283000F5E701462B4642463846FFF7D0FE0446F0
:1028400008B93046E7E7054B0146B3F9000000F050
:1028500078FA0028E9DD02B0BDE8F081700F0020B1
:102860002DE9F041437F23F007030B43052904467C
:10287000437720D0072903D004294BD1264E05E009
:10288000B0F91E00FFF770F9D0F8F060234B04F1A7
:102890003C05B3F900702846FDF7D6FF40F2172338
:1028A000A4F8523004F150023B4631462846BDE8B8
:1028B000F04100F041BEB0F91E00FFF755F90323C7
:1028C000064684F87430231D1A4606F1E005B4F973
:1028D0001E000021FFF786FF01212846FEF708FDB4
:1028E0000E4BD6F8F470B3F9008004F13C06304684
:1028F000FDF7AAFF40F21223A4F8523030464346B7
:1029000004F15002394600F017FE2846BDE8F041B8
:10291000FEF71EBDBDE8F081404B4C00700F00205B
:10292000F8B51E469F1C5B780446154608461BB941
:102930006FF015042046F8BD10221649083001F04A
:1029400089FC0028F4D01CB9853D022D0FD908E080
:1029500094F91030013307D1A368853D022D1C780E
:1029600004D96FF08504E5E76468ECE754B973783F
:1029700008226FF0010412FB034403FB026313F807
:10298000012D2AB122463946069801F072FCD1E7A2
:10299000013CF4E7C652000870B51D465B7804465A
:1029A0001646084613B96FF0150070BD1022124983
:1029B000083001F04FFC0028F5D0882E1AD1A91C50
:1029C00034B194F91030013310D1A3681C783CB9AC
:1029D0006C78E408023CE4B20B1913F8013C3BB1FB
:1029E0002246049801F045FC204670BD6468E7E784
:1029F000013CF0E7002070BDC6520008F8B517464C
:102A00000D46FFF7B1F87C78012C064610D1862DD3
:102A10000CD100F1E00521462846FEF769FC7B68F1
:102A20001BBAA6F8E8302846FEF792FC2046F8BD0F
:102A30000020F8BDF0B55378042B87B00646144645
:102A400038D1862902D0012007B0F0BD02F110076D
:102A500031490822384601F0FDFB0028F3D0237CE1
:102A6000FF2B04D1637C03F00F03022BEBD039461C
:102A70003046FFF7B9F8054618B1427CA3789A4270
:102A800025D063681BB31022002102A801F0FCFBD3
:102A9000E3785A0610D4A278394602A800F04FFC19
:102AA000E378A27803F0C00302A93046FFF766F886
:102AB000054660B90020C7E708230093002204AB55
:102AC0000721304600F057F90028E4DAF2E76168A0
:102AD00031B9002DB7D029463046FFF775F8B2E777
:102AE000A36809BA1BBAAB614B1C69610AD00B4BD6
:102AF0000B481B8841431BB205F1300205F11C0055
:102B000000F01AFD2B7CE27823F07F0322F03F02D5
:102B100013432B7497E700BF9652000890020020E1
:102B200040420F002DE9F047984688B006460F4610
:102B30001446002308226949DDF84090039340467B
:102B400001F088FBA8B198F80030FF2B05D198F868
:102B5000013003F00F03022B0BD0414604BB03A846
:102B6000FFF774F80446039B33B193F91030002B40
:102B700002DAB8F1000F04D1FFF784FD002818BF76
:102B800080464146204601F03DF8054668B1417F48
:102B900001F007014B1E012B00F2938000209AE008
:102BA0002046FFF779F80390DDE702230093024601
:102BB00003464146204600F0D1FF05460028EDD0EF
:102BC000474E73680BB9376827B1F368C3B9B36868
:102BD000B3B9012706EBC70A0121CAF80490484699
:102BE00000F018FB002346F837302B681BB9C5F8F6
:102BF00000A005E013461A68002AFBD1C3F800A024
:102C0000002340F2FF22CDE904234FF080730693A6
:102C1000FF238DF81C3098F80D308DF81D30B8F872
:102C20000E30ADF81E301CBB02AE304600F0BCF8D2
:102C30000746BC4213D12B4B05F13C04B3F90060AD
:102C40002046FDF701FE40F21223A5F8523005F1AF
:102C5000500233462449204600F06EFC9EE736F9C8
:102C6000140004AB42460021FFF7BCFD0134E0E74D
:102C70002046FEF779FF0646424604AB2046002177
:102C800006F1E004FFF7AEFD01212046FEF730FB20
:102C9000144BD6F8F470B3F9008005F13C063046C9
:102CA000FDF7D2FD40F21223A5F8523030464346DC
:102CB00005F15002394600F03FFC2046FEF748FB84
:102CC0006CE7032902D10421FFF7CAFD2A463946E1
:102CD000304600F0DFFF08B0BDE8F08796520008EC
:102CE0008C100020700F002040420F002DE9F341AE
:102CF0000446884617461E4600F0B6F8054648B119
:102D00004146204600F09EF8691E0446304600F019
:102D100081FA1CB9284602B0BDE8F081B4F9081068
:102D2000ADF802706846019600F02EFD002803DC25
:102D30000021304600F080FA204600F0A9F8044651
:102D4000E7E707B540F20223019101466846ADF876
:102D5000023000F019FD03B05DF804FB07B540F246
:102D60000123019101466846ADF8023000F00CFDE8
:102D700003B05DF804FB00B589B006930A9BADF87B
:102D80001C304FF401738DF81410ADF81620ADF817
:102D90000630024605AB03A901A8029300F018FD16
:102DA000049809B05DF804FB044BB3F9003013B18B
:102DB0000380012070471846704700BF9C10002018
:102DC0002DE9F041174603F108020A440E4600219E
:102DD00080461C4608464FF0FF3300F04FF9054689
:102DE000E8B18068002306704470438043718371AA
:102DF0000371B8F1000F05D026B1324641460830C4
:102E000001F037FA5FB154B1A8684378A34206D104
:102E10000378083322463946184401F02AFA284636
:102E2000BDE8F081C3B2022B9FBF054B53F82020B1
:102E30000A6043F8201094BF00206FF0150070471F
:102E4000A0100020C3B2022B09D8064B53F8200073
:102E500000B9704743688B4202D00068F8E7002051
:102E6000704700BFA0100020C3B2022B0BD8074B45
:102E700053F82030002003B970475A681B688A4213
:102E800008BF0130F7E70020704700BFA010002006
:102E900028B14368006810B142689342FAD1704784
:102EA00029B190F91030022B04D100F080BD6FF0F1
:102EB000150070476FF00100704700B9704790F936
:102EC00010308B42FAD04068F7E7000030B5034677
:102ED000154A072B88BF033310688CBF23F0030308
:102EE00008230021F8B14468A3420ED8E41A072C45
:102EF0000ED90E4D03445D1BB5F5007F0ED90021A0
:102F00001160026883E8140030BD01460068E9E7FB
:102F1000036809B9136030BD0B6030BD09B9136097
:102F2000EFE70B60EDE730BDAC100020AC100020E7
:102F30001D4BC31AB3F5007F30B533D21B4C22684A
:102F400000230AB1824211D307298ABF0331082125
:102F500021F00301164D02604218AA1A072A98BFF1
:102F6000891841602BB9206003460EE013461268B1
:102F7000E7E75A6818601A44821A072AF4D80268E8
:102F80001A604268C11A0A445A601A6852B15968F4
:102F90001944511A072905D811681960D11A5268C5
:102FA0000A445A6030BD00BFB4100020AC100020AD
:102FB000B41200202DE9F843814614200F4616462E
:102FC0009846FFF783FF044650B166B13046FFF7DD
:102FD0007DFF054640B920461421FFF7A9FF2C4686
:102FE0002046BDE8F88335460123C4F80490A56067
:102FF000E66084F810802360002FF1D03246394615
:10300000284601F036F9EBE770B50446002504B90F
:1030100070BD94E84800012B0AD1E168A0682560E2
:10302000FFF786FF14212046FFF782FF3446EEE7C4
:10303000013B2360FAE7000001210148FEF758B97F
:10304000B010002008B5FFF7F7FF094A094B1360DD
:10305000022100221A705A709A70DA701A7159712E
:103060009A71DA710448BDE80840FEF771B900BFF3
:10307000AC100020B4100020B0100020B2F5007F8A
:10308000F8B505460E4614461F460DD8FFF7D4FF87
:1030900022463B4631462846FFF78CFF044603484C
:1030A000FEF756F92046F8BD0024FBE7B0100020DB
:1030B00007292DE9F84388BFCF1C0D468CBF27F0A8
:1030C0000307082704469146FFF7B6FF2DB124B148
:1030D000E3689D4201D8A36833B92A48FEF738F95E
:1030E00000263046BDE8F8831420FFF7EFFE0646C1
:1030F0000028F2D0E3689D423DD0AF4202D85A1B6F
:10310000072A38D82846FFF7E1FE074620B91421E0
:103110003046FFF70DFFE0E7E068401BFFF7D6FE03
:10312000804630B914213046FFF702FF2946384661
:10313000EFE72A46A168384601F09BF8E268A168EB
:10314000521B2944404601F094F8E168A068FFF75B
:10315000EFFEC4F80880E3680A485B1BE36063681D
:1031600073600123B760F56086F810903360666085
:10317000FEF7EEF8B5E7A7689D4214BF7B19002360
:10318000A360E8E7B010002070B50729044688BFA7
:10319000CE1C0D468CBF26F003060826FFF74CFF19
:1031A000E3689D4204D11A48FEF7D2F8002070BDB2
:1031B0003DB9A06838B11946FFF7BAFEA560E560D1
:1031C000F1E79D4202D8991B072917D82846FFF737
:1031D0007DFE064620B90E48FEF7BAF80C2070BDF9
:1031E000A16829B1E268AA4228BF2A4601F041F845
:1031F000E168A068FFF79CFEA660E0E7033323F0D8
:1032000003039E42DBD2A0683044FFF791FED6E76D
:10321000B010002038B504460D46FFF70DFF24B965
:103220000448BDE83840FEF793B823682B44236078
:103230006468F4E7B010002010B50446FFF7FCFE08
:103240002046FFF7E1FE0248BDE81040FEF780B8D7
:10325000B010002038B50446FFF7EEFE0CB1E2686E
:103260002AB90E48FEF774F80025284638BD2368B1
:10327000012B0ED994F91030A1686068FFF79AFE0F
:10328000054610B12368013B23600448FEF760F84F
:10329000EBE70248FEF75CF82546E6E7B0100020B1
:1032A00010B504468C42084606D16468002141608E
:1032B000FFF7C2FF204610BD23465A68002AF5D00A
:1032C000904202D142685A60F0E71346F5E730B504
:1032D0004B68456804680A689D4208BF944209D15A
:1032E000C568CB6884688A689D4206BF9442012005
:1032F000002030BD002030BD30B5F8B1D9B18842D2
:103300001BD0421E0139002012F8013F11F8015F65
:10331000AB4200F1080403D1E0B28028F4D130BD03
:103320006B40E4B21A0609D40130C0B25B00A0427F
:10333000DBB2F7D130BD084630BD802030BD802AD9
:1033400028BF8022F8B5D50814462A4606460F46FF
:1033500000F08FFF63070ED0A4EBC504FF23C4F178
:10336000080403FA04F4735D23EA040373557A5DD9
:10337000144023437355F8BD2DE9F04706468AB043
:1033800020B9002630460AB0BDE8F0870029F8D001
:1033900000274FF0FF333D463C46184631F817E012
:1033A000BEF1000F12D1B3F1FF3F13BF01353BB2A5
:1033B00001252DB20137082FF0D15F1C13D0471C17
:1033C00001D0AC4211DA2C4618460EE0B3F1FF3FB3
:1033D000F0D0B0F1FF3F01D0AC4201DA2C461846E4
:1033E0004FF0FF33E6E7451C03D0012CD8BF4FF068
:1033F000FF30394F00256B46EC464FF03A09A842A2
:103400001AD183F800900519072D03F10103F6DDA9
:10341000411C05D02044082802BF3A21197001330D
:10342000002103F8011BA3EB0C039342A9D86146CA
:10343000304600F0ADFFA5E715B183F800900133E9
:1034400011F815E01EF0F00F4FEA450821D04FEAC1
:103450001E1A0EF00F0E17F80AA017F80EE083F8E8
:1034600001E001EB080E83F800A09EF801E04FEAAE
:103470001E1E033317F80EE003F801EC88440135F3
:1034800098F801E00EF00F0E17F80EE083F800E058
:10349000BAE7BEF1000F10D017F80EA09E460EF846
:1034A00002AB01EB080A9AF801A04FEA1A1A17F8C2
:1034B0000AA083F801A07346E0E701EB080E9EF82E
:1034C00001E01EF0F00F1FBF4FEA1E1E17F80EE0BE
:1034D00083F800E00133D1E7D65200080C4B30B539
:1034E00018680C4CA0FB0445EA0B4AF6C85101FBD6
:1034F00012004BF68F41414340F6475000FB121239
:1035000012B11A60186830BD6FF00042F9E700BFD1
:103510002402002091138FBC10B5FFF7DFFF044693
:10352000FFF7DCFFE413C0F3CF3040EA044010BDE6
:10353000B0F9001000F004B930B4034DC560026169
:1035400030BC1380FDF792B931350008F8B5054657
:103550000E46FCF77BFF364B364A1B881BB20746EC
:1035600052F823301A6A002A4ED05C699969A14248
:103570004AD9611C5961D9690C4046B9196931B9F8
:10358000611C04D13846FCF769FF2046F8BD002CC9
:103590003EDB02EBC40103C985E803001E69002E6F
:1035A00038D031681961002C1EDA736893E8030083
:1035B00085E8030016F8043C052B23D00023736034
:1035C0000A21A6F10800FCF751FE16F8034C384614
:1035D000FCF744FF0E2C28D82046FCF787FE24E099
:1035E0003846FCF73BFF20E09D695969D869691AA4
:1035F0008842A9BF691C4FF0FF350540996102EB75
:10360000C505D2E70F24E2E74FF0FF34002EB5D016
:10361000DD60C3E7002CE3DA18460321FCF726FE41
:103620003846FCF71BFFFCF7DBFE0124ADE700BFCB
:1036300090020020E002002010B583694469C2694D
:103640001C1BA24201DA002010BD5C1C13408461E7
:10365000F9D4026A03C902EBC30383E80300012023
:1036600010BD00002DE9F8431E46264B53F82150AB
:10367000254B1B880380074691463DB93046FCF731
:10368000EDFE4FF0FF342046BDE8F8832B79032B85
:103690002ED01E4B01462846D3F80080FFF7CCFF02
:1036A000044650B13046FCF7D9FE98F80430052B9B
:1036B00001D1FCF795FE0124E5E7B9F1000F03D134
:1036C0003046FCF7CBFEDEE798F80430C8F80C7003
:1036D000052B0CBF052104214046FCF7C7FD4146E0
:1036E00005F11000FDF774F93046FCF7B7FEE0E78E
:1036F00003C8EB6883E803000A212846FCF7B6FDFF
:10370000F2E700BFE00200209002002094020020B7
:1037100038B50446FCF79AFE074B1B882380074BFD
:10372000214605461868FFF787FF04462846FCF740
:1037300095FE204638BD00BF900200209402002074
:1037400008B50F4B53F82130B3B1212202801A790A
:10375000032A0BD103C8DA6882E8030018460A215D
:10376000FCF784FD074B0120186008BD0146184690
:10377000BDE80840FFF760BF4FF0FF3008BD00BF55
:10378000E00200209802002070B504460D46FCF7C8
:1037900068FE064628B129462046BDE87040FFF77E
:1037A000CFBF0A4B1B881BB29D4204D12046BDE807
:1037B0007040FFF7ADBFFCF749FE3246034629468D
:1037C0002046BDE87040FFF74DBF00BF90020020CB
:1037D0002DE9F0410C4617460546FCF737FE0C4B29
:1037E0001A880C4B12B2804653F8226005213046ED
:1037F000FCF73CFD95E80300F460434684E80300D1
:10380000012239462046BDE8F041FFF72BBF00BF3B
:1038100090020020E002002070B504460D46FCF73F
:1038200015FE104BB4F9002053F822402379052BE4
:10383000064604D0FCF712FE4FF0FF3070BD95E84D
:103840000300E36883E803000A212046FCF70EFD2D
:1038500064793046FCF702FE2046FCF747FD012064
:1038600070BD00BFE00200200121FFF76FBE000025
:10387000044B1B680022013918625A619A61D961B0
:10388000704700BF94020020F8B5064684890F46B1
:1038900015460020ADB90023B289B16800F00FFAD7
:1038A0004FF6C57302199A42396816DC3A3420443F
:1038B00000232022083180B200F001FAC04380B218
:1038C000F8BDAE42E7D02346AA89A96800F0F7F90F
:1038D000EB686D681C44A4B2DCE7013080B2E5E718
:1038E0002DE9F3410C46804602212046FFF7E5FA18
:1038F00005460121FFF7E1FAEB68032B074643D9A0
:1039000000F1080122462846AE68FFF7BDFF0028F7
:103910003AD13378803B082B0CD8DFE803F0050B55
:103920000B0B0B0B1A232C00AB89B96832464046AF
:1039300000F076F83178234640F201220220FFF7AA
:10394000D5F9014600BB204602B0BDE8F041FFF7C3
:1039500073BCEB680093BA68334621464046FEF7D5
:103960006BFCE7E7EB680093BA68334621464046B4
:10397000FEF71EFBDEE7EB680093BA68334621468C
:103980004046FEF77BFBD5E702B0BDE8F08138B5D5
:103990000D46144600211A460223FFF76FFB28B19B
:1039A000836800221D705C709A70DA7038BD10B5A3
:1039B000044668B190F91030022B0CD142680831EE
:1039C000FFF762FF50B1A36840BA5880002010BDD5
:1039D0006FF00D0010BD6FF04C0010BD6FF00100D6
:1039E00010BD2DE9F041DDF81880154600220E4685
:1039F0001F46014608F108031046FFF7C8FF0446BA
:103A000050B1806876BA6DBA8680C58027B14246CB
:103A10003946083000F02DFC2046BDE8F08100005A
:103A2000F7B506460C46002A38D0072B36D99188C0
:103A3000D088083B40BA49BA009389B202F1080322
:103A400082B28120FFF7CDFF074638B3237EFF2BDC
:103A500004F108020CBF002104F1180100F022F863
:103A6000054630B90146384603B0BDE8F040FFF7DF
:103A7000E3BB00231A4619461846FFF7A1F98368ED
:103A800007495E8004464560034640F20222012059
:103A9000FFF72CF9014608B92046E5E703B0F0BD71
:103AA0000000FFFFF8B50F4616460123282200212B
:103AB000FFF7E4FA0546A0B18468102204F108007B
:103AC000394687B100F0D5FB04F1180010223146C9
:103AD00066B100F0CEFB60232360FF23A3710023B7
:103AE000E3712846F8BD00F0CFFBEDE700F0CCFB1A
:103AF000012384F82730EEE708B51022034900F0CF
:103B0000A9FBB0FA80F0400908BD00BFC65200080A
:103B100070B50446002625689DB904F12000FCF725
:103B200093FE04F13C00FCF78FFE04F15800FCF713
:103B30008BFE10222946201D00F0A6FB6577E58349
:103B400070BD00216868FFF777FB23685E60002B7B
:103B5000E1D01A6822601E60DDE700002DE9F84F11
:103B6000834690461E469DF82870894619B9002460
:103B70002046BDE8F88F082BF9D80846FFF7BCFFB0
:103B80000028F4D11E4C4946201DFFF7A0FB254616
:103B9000824638BB201DFFF7AFFF0028E7D0204644
:103BA000A4F81EB040F804AB1022494600F061FBB7
:103BB000B8F1000F07D036B13246414605F1140086
:103BC00000F057FB2E776F7707F00707022F04BF2F
:103BD000032385F874304FF40473EB86AD636D6591
:103BE000074CC5E7B8F1000FC2D0002EC0D0324656
:103BF000414604F1140000F03CFB26776777B7E7F5
:103C0000B412002038B505460C4661B10846FFF7EE
:103C100073FF40B9084BB3F91E3033B9214607484A
:103C2000FFF755FB30B9002038BD002DF6D09D427E
:103C3000F9D1F3E7004838BDB4120020B8120020D3
:103C400008B5FFF7DFFF18B1BDE80840FFF760BF18
:103C500008BD000038B538B100F17804074DAC421A
:103C600004D30024204638BD054CF7E7201DFFF79C
:103C700043FF0028F6D07834F1E700BF2C13002072
:103C8000B412002008B5FFF7E5FF10B1437F1B0712
:103C9000F9D508BD10B514462AB1537F03F00703C8
:103CA000013B012B01D8002010BD137F0B70127F48
:103CB00004F1140100F0DDFAB4F91E0010BDF0B5F6
:103CC000CAB1DC0705D511F8014B013A204492B284
:103CD0000133570801EB47054C1C03350234AC4255
:103CE0000AD11A44D30703D511F8173000EB03208B
:103CF000030C09D180B2F0BD14F803EC14F8026C87
:103D000006EB0E263044E9E713FA80F0F0E70000F6
:103D100080F0004002E000BF81F0004142001FBF80
:103D20005FEA410392EA030F7FEA226C7FEA236C89
:103D30006AD04FEA1262D2EB1363C1BFD21841407E
:103D400048404140B8BF5B42192B88BF704710F014
:103D5000004F40F4000020F07F4018BF404211F0B7
:103D6000004F41F4000121F07F4118BF494292EA1F
:103D7000030F3FD0A2F1010241FA03FC10EB0C004B
:103D8000C3F1200301FA03F100F0004302D54942D8
:103D900060EB4000B0F5000F13D3B0F1807F06D385
:103DA00040084FEA310102F10102FE2A51D2B1F17D
:103DB000004F40EBC25008BF20F0010040EA030072
:103DC0007047490040EB000010F4000FA2F101021F
:103DD000EDD1B0FA80FCACF1080CB2EB0C0200FAA9
:103DE0000CF0AABF00EBC25052421843BCBFD040F7
:103DF0001843704792F0000F81F4000106BF80F471
:103E000000000132013BB5E74FEA41037FEA226C33
:103E100018BF7FEA236C21D092EA030F04D092F0FE
:103E2000000F08BF0846704790EA010F1CBF002032
:103E3000704712F07F4F04D1400028BF40F000408F
:103E4000704712F100723CBF00F50000704700F0AF
:103E5000004343F0FE4040F4000070477FEA2262D6
:103E600016BF08467FEA23630146420206BF5FEAA7
:103E7000412390EA010F40F4800070474FF00003A7
:103E800004E000BF10F0004348BF40425FEA000C6E
:103E900008BF704743F0964301464FF000001CE016
:103EA00050EA010208BF70474FF000030AE000BF6C
:103EB00050EA010208BF704711F0004302D54042AA
:103EC00061EB41015FEA010C02BF8446014600201C
:103ED00043F0B64308BFA3F18053A3F50003BCFA37
:103EE0008CF2083AA3EBC25310DB01FA02FC6344E4
:103EF00000FA02FCC2F12002BCF1004F20FA02F2EB
:103F000043EB020008BF20F00100704702F12002DD
:103F100001FA02FCC2F1200250EA4C0021FA02F23E
:103F200043EB020008BF20EADC7070474FF0FF0C43
:103F30001CEAD0521EBF1CEAD15392EA0C0F93EA3E
:103F40000C0F6FD01A4480EA010C400218BF5FEAE0
:103F500041211ED04FF0006343EA501043EA511153
:103F6000A0FB01310CF00040B1F5000F3EBF49004D
:103F700041EAD3715B0040EA010062F17F02FD2A51
:103F80001DD8B3F1004F40EBC25008BF20F0010034
:103F9000704790F0000F0CF0004C08BF49024CEA4B
:103FA000502040EA51207F3AC2BFD2F1FF0340EADD
:103FB000C250704740F400004FF00003013A5DDC4E
:103FC00012F1190FDCBF00F000407047C2F100028F
:103FD000410021FA02F1C2F1200200FA02FC5FEA7C
:103FE000310040F1000053EA4C0308BF20EADC70C6
:103FF000704792F0000F00F0004C02BF400010F438
:10400000000F013AF9D040EA0C0093F0000F01F0E4
:10401000004C02BF490011F4000F013BF9D041EA06
:104020000C018FE70CEAD15392EA0C0F18BF93EA08
:104030000C0F0AD030F0004C18BF31F0004CD8D132
:1040400080EA010000F00040704790F0000F17BFB9
:1040500090F0004F084691F0000F91F0004F14D0FF
:1040600092EA0C0F01D142020FD193EA0C0F03D157
:104070004B0218BF084608D180EA010000F000405A
:1040800040F0FE4040F40000704740F0FE4040F435
:10409000400070474FF0FF0C1CEAD0521EBF1CEAD4
:1040A000D15392EA0C0F93EA0C0F69D0A2EB0302F2
:1040B00080EA010C49024FEA402037D04FF080538C
:1040C00043EA111143EA10130CF000408B4238BF51
:1040D0005B0042F17D024FF4000C8B4224BF5B1A5F
:1040E00040EA0C00B3EB510F24BFA3EB510340EAAD
:1040F0005C00B3EB910F24BFA3EB910340EA9C005B
:10410000B3EBD10F24BFA3EBD10340EADC001B01CA
:1041100018BF5FEA1C1CE0D1FD2A3FF650AF8B426E
:1041200040EBC25008BF20F0010070470CF0004C7B
:104130004CEA50207F32C2BFD2F1FF0340EAC250A6
:10414000704740F400004FF00003013A37E792F067
:10415000000F00F0004C02BF400010F4000F013AC5
:10416000F9D040EA0C0093F0000F01F0004C02BFC0
:10417000490011F4000F013BF9D041EA0C0195E729
:104180000CEAD15392EA0C0F08D142027FF47DAFC2
:1041900093EA0C0F7FF470AF084676E793EA0C0FB2
:1041A00004D14B023FF44CAF08466EE730F0004CB0
:1041B00018BF31F0004CCAD130F000427FF45CAF40
:1041C00031F000437FF43CAF5FE700BF42000ED206
:1041D000B2F1FE4F0BD34FF09E03B3EB126209D442
:1041E0004FEA002343F0004323FA02F070474FF0F8
:1041F0000000704712F1610F01D1420202D14FF06D
:10420000FF3070474FF00000704700BF70B50D4E93
:104210000D4CA41BA4100025A54209D10B4E0C4C3B
:10422000FBF7B2FFA41BA4100025A54205D170BD69
:1042300056F8253098470135EEE756F8253098476F
:104240000135F2E7705300087053000870530008FE
:104250007053000810B501390244904201D100208A
:1042600010BD10F8013B11F8014FA342F5D0181B07
:1042700010BD10B5431E0A44914200D110BD11F883
:10428000014B03F8014FF7E702440346934200D184
:10429000704703F8011BF9E70FB40A4B13B51C680C
:1042A00024B1A36913B9204600F02CFA05AB049A97
:1042B000A1680193204600F0E3FB02B0BDE8104086
:1042C00004B070472802002070B50E46054618B1AC
:1042D00083690BB900F016FAAB69AC6813B92846CC
:1042E00000F010FA234B9C4217D16C68A3891B077E
:1042F0001DD52369DBB1013EA36816F8011F013B00
:10430000A360E9B9002B2EDA22460A21284600F0E4
:1043100047F8013011D00A2070BD174B9C4201D1E3
:10432000AC68E3E7154B9C4208BFEC68DEE721462A
:10433000284600F087F80028DDD04FF0FF3070BD30
:10434000002B04DAA269934206DB0A2904D0236811
:104350005A1C22601970CFE72246284600F020F848
:104360000130C9D1E9E723680A205A1C226018707D
:1043700070BD00BF0C5300082C530008EC5200081D
:10438000024B01461868FFF79FBF00BF28020020BC
:10439000034611F8012B03F8012B002AF9D17047CD
:1043A000F8B50E461446054618B183690BB900F0FE
:1043B000A9F9214B9C422AD16C68A369A360A38907
:1043C0001A072ED5236963B323692068C01A63696D
:1043D000F6B29842374604DB2146284600F028F919
:1043E00028BBA368013BA36023685A1C22601E708F
:1043F00063690130984204D0A389DB0719D50A2EDE
:1044000017D12146284600F013F990B10FE00B4B6D
:104410009C4201D1AC68D0E7094B9C4208BFEC68D4
:10442000CBE72146284600F00DF80028CCD04FF00D
:10443000FF373846F8BD00BF0C5300082C53000866
:10444000EC520008324B70B51D6806460C4625B18B
:10445000AB6913B9284600F055F92E4B9C420FD199
:104460006C68B4F90C309AB215072CD4D00611D46C
:104470000922326043F04003A3814FF0FF3070BD4A
:10448000254B9C4201D1AC68EBE7244B9C4208BF12
:10449000EC68E6E7510712D5616B41B104F14403C2
:1044A000994202D0304600F017FA00236363A389D3
:1044B00023F02403A3810023636023692360A3897D
:1044C00043F00803A38123694BB9A38903F4207344
:1044D000B3F5007F03D02146304600F0C1F9A28930
:1044E00012F001030CD00023A36063695B42A36157
:1044F000236953B9B4F90C3013F08000BAD170BD00
:10450000920758BF6369A360F2E70020F7E700BF96
:10451000280200200C5300082C530008EC5200081D
:104520008A892DE9F041054610070C465AD44B689C
:10453000002B05DC0B6C002B02DC0020BDE8F081B9
:10454000E66A002EF9D0002312F480522F682B6007
:1045500033D0606DA3895A0705D56368C01A636BB1
:104560000BB1236CC01A00230246E66A216A284672
:10457000B047431CA38906D129681D294BD82B4A73
:10458000CA40D60747D500226260D904226922605A
:1045900004D5421C01D12B6803B96065616B2F60A3
:1045A0000029CAD004F14403994202D0284600F001
:1045B00093F900206063BDE8F081216A0123284659
:1045C000B047411CC6D12B68002BC3D01D2B01D096
:1045D000162B01D12F60B0E7A38943F04003A381DC
:1045E000BDE8F0810F69002FA7D093070E6808BFC0
:1045F0004B690F6018BF0023A6EB07088B60B8F16A
:10460000000F9ADD43463A46216AA66A2846B0471B
:10461000002807DCA38943F04003A3814FF0FF305B
:10462000BDE8F0810744A8EB0008E8E7010040205E
:1046300038B50B6905460C46DBB118B183690BB977
:1046400000F060F80C4B9C4209D16C68B4F90C3056
:104650007BB121462846BDE83840FFF761BF074BD4
:104660009C4201D1AC68F1E7054B9C4208BFEC6865
:10467000ECE7002038BD00BF0C5300082C530008A5
:10468000EC520008014900F0A9B800BF314600080B
:10469000002310B504460360436083608181436654
:1046A000C281036143618361194608225C30FFF7D0
:1046B000EBFD054B6362054BA362054BE362054BC3
:1046C0002462236310BD00BFD94F0008FB4F0008D0
:1046D000335000085750000870B54A1E68255543EE
:1046E0000E4605F1740100F045F9044640B1002181
:1046F00080E842000C30A06005F16802FFF7C4FDBD
:10470000204670BD836910B5044633BB8364C3641F
:104710000365124B124A1B688262984204BF012350
:10472000836100F01FF86060204600F01BF8A06075
:10473000204600F017F80022E06004216068FFF7CF
:10474000A7FF01220921A068FFF7A2FF0222122180
:10475000E068FFF79DFF0123A36110BDE852000848
:1047600085460008F8B51C4B1E68B369074613B9A7
:104770003046FFF7C7FF4836B4687368013B03D57E
:10478000336833B13668F7E7B4F90C506DB168346B
:10479000F4E704213846FFF79FFF30600028F1D18D
:1047A0000C233B6004462046F8BD4FF6FF73E381BF
:1047B0000123A38165662560A5606560256165614B
:1047C000A5610822294604F15C00FFF75DFD6563E1
:1047D000A563A564E564E6E7E85200082DE9F8431F
:1047E0008046894600F14804002614B93046BDE8E9
:1047F000F883A5686768013F01D52468F5E7AB89B0
:10480000012B07D9B5F90E30013303D029464046B4
:10481000C84706436835EEE770B50E46B1F90E108D
:10482000002990B014461D4607DA00232B60B38997
:104830001A0610D44FF480630EE001AAFBF7D8FCEF
:104840000028F2DB029A02F47042A2F500535A42A9
:104850005A412A60EEE740230020236010B070BD6B
:104860008B8973B59D0706460C4607D504F14703AF
:10487000236023610123636102B070BD01AB6A460E
:10488000FFF7CAFF00990546304600F073F838B9C3
:10489000B4F90C309A05EFD443F00203A381E5E7A5
:1048A0000C4BB362A389206043F08003A381009B7B
:1048B0006361019B20614BB1B4F90E103046FBF7E8
:1048C0009CFC18B1A38943F00103A381A3891D4374
:1048D000A581D1E78546000838B50546002945D0B1
:1048E00051F8043C0C1F002BB8BFE41800F008FC82
:1048F0001F4A1368104633B9636014602846BDE848
:10490000384000F0FEBBA3420CD9216862189342E4
:1049100004BF1A685B68636004BF521822600460B9
:10492000ECE713465A680AB1A242FAD91968581836
:10493000A0420BD120680144581882421960DDD191
:10494000106852685A6001441960D7E702D90C23F5
:104950002B60D3E7206821188A4204BF116852688F
:10496000626004BF091821605C60C7E738BD00BF02
:104970002C13002070B5CD1C25F0030508350C2D37
:1049800038BF0C25002D064601DBA94203D90C23B4
:104990003360002070BD00F0B3FB234A1468214649
:1049A00091B9224C23681BB93046FBF7F1FB20601C
:1049B00029463046FBF7ECFB431C26D10C23336021
:1049C000304600F09EFBE4E70B685B1B1AD40B2B10
:1049D0000FD90B60CD50CC18304600F092FB04F19B
:1049E0000B00231D20F00700C31A1BD05A42E250CF
:1049F00070BD8C420DBF63684B686360136018BF65
:104A00000C46E9E70C464968CAE7C41C24F00304D5
:104A1000A04205D0211A3046FBF7BAFB0130CDD0B9
:104A20002560D9E770BD00BF2C1300203013002093
:104A30009368013B002B10B4936008DA9469A34299
:104A400002DBCBB20A2B02D110BCFFF7A9BC136862
:104A5000581C10601970C8B210BC7047F8B50646F3
:104A60000F461446D518AC4201D1002007E03A4663
:104A700014F8011B3046FFF7DBFF431CF3D1F8BDF0
:104A80002DE9F04F9DB00C4617460393064618B12A
:104A900083690BB9FFF736FE7C4B9C4257D1746893
:104AA000A38918075DD52369002B5AD000230993E9
:104AB00020238DF8293030238DF82A304FF0010B58
:104AC000B846454615F8013B002B55D1B8EB070A0F
:104AD0000BD053463A4621463046FFF7BFFF013020
:104AE00000F0C480099B5344099398F80030002BD0
:104AF00000F0BC8000234FF0FF320493079305922F
:104B000006938DF853301A9305222978604800F0F7
:104B1000A7FA05F10108049B002831D1D90644BF4A
:104B200020228DF853201A0744BF2B228DF85320E2
:104B30002A782A2A2CD0079A00210A20A846013573
:104B400098F80030303B092B6DD971B326E0514BFA
:104B50009C4201D1B468A3E74F4B9C4208BFF46864
:104B60009EE721463046FFF76DFC00289ED04FF0AF
:104B7000FF301DB0BDE8F08F252BA7D0A846A0E7D9
:104B8000434A801A0BFA00F0184304904546BBE7ED
:104B9000039A111D12680391002A01DB079204E0B9
:104BA000524243F002030792049398F800302E2BF0
:104BB00010D198F801302A2B08F1010137D1039B5D
:104BC0001A1D1B680392002BB8BF4FF0FF3308F18A
:104BD00002080593314D98F800100322284600F092
:104BE0003FFA40B14023401B03FA00F0049B03430B
:104BF000049308F1010898F8001029488DF828104E
:104C0000062208F1010700F02BFA002834D0254BCA
:104C100003BB039B073323F0070308330393099B6C
:104C20004B4409934CE700FB0232012186E7002345
:104C3000059318460A258846013198F80020303A35
:104C4000092A03D9002BC5D00590C3E705FB002036
:104C50000123F0E703AB00932246134B04A930462F
:104C6000AFF30080B0F1FF3F8146D8D1A3895B0646
:104C70003FF57DAF09987CE703AB009322460A4BD2
:104C800004A9304600F088F8ECE700BF0C53000898
:104C90004C5300082C530008EC52000852530008F3
:104CA00056530008000000005D4A00082DE9F04757
:104CB00091461F468A680B69DDF820809342B8BF91
:104CC0001346C9F8003091F8432006460C4612B14D
:104CD0000133C9F800302368990642BFD9F8003083
:104CE0000233C9F80030256815F0060507D104F134
:104CF000190AE368D9F800209B1A9D4229DB94F831
:104D000043302268003318BF012392062ED404F1E9
:104D1000430239463046C047013021D02368E56858
:104D2000D9F8002003F00603042B08BFAD1AA368CE
:104D300022690CBF25EAE57500259342C4BF9B1A82
:104D4000ED184FF000091A344D451BD10020BDE885
:104D5000F0870123524639463046C047013003D11F
:104D60004FF0FF30BDE8F0870135C2E7E1185A1C6B
:104D7000302081F84300224494F8451082F8431013
:104D80000233C4E70123224639463046C04701308A
:104D9000E6D009F10109D7E72DE9F04317460A7E6D
:104DA00085B06E2A984606460C460C9B01F1430ED0
:104DB00000F0BC801AD8632A2ED00AD8002A00F04E
:104DC000C880582A00F08A8004F1420584F8422005
:104DD0002AE0642A01D0692AF6D121681A6811F004
:104DE000800F23D0111D1960136827E0732A00F08B
:104DF000B48008D86F2A2AD0702AE5D10A6842F018
:104E000020020A6003E0752A21D0782ADCD17822BA
:104E100084F845206E4964E01A6801F14205111DCD
:104E20001960136884F842300123A3E011F0400FA9
:104E300002F104011960D7D0B2F90030002B03DA77
:104E40002D225B4284F8432062490A2217E0206841
:104E5000196810F0800F03D0081D18600B6806E079
:104E600010F0400F01F104001860F7D00B88594989
:104E70006F2A14BF0A220822002084F843006568C4
:104E8000A560002DC0F29C80206820F00400206006
:104E9000002B3FD1002D40F095807546082A0BD19C
:104EA0002368DA0708D5236962689A42DEBF302397
:104EB00005F8013C05F1FF35AEEB05032361CDF8A4
:104EC00000803B4603AA21463046FFF7EFFE013043
:104ED00055D14FF0FF3005B0BDE8F08381F8452093
:104EE0003C492268186812F0800F00F104051D602B
:104EF00001D0036802E05506FBD50388D00744BF04
:104F000042F0200222601BB9226822F020022260B7
:104F10001022B1E77546B3FBF2F002FB1033CB5C15
:104F200005F8013D03460028F5D1B7E708681A687F
:104F3000496910F0800F04D0101D186013681960C3
:104F400007E010F0400F02F1040018601368F6D07B
:104F50001980002323617546B1E71A68111D196095
:104F6000156862680021284600F07AF808B1401BF5
:104F7000606063682361002384F843309FE72369FE
:104F80002A4639463046C0470130A2D023689B07E5
:104F900007D5002504F11909E368039A9B1A9D427D
:104FA00005DBE068039B9842B8BF184693E70123EE
:104FB0004A4639463046C04701308AD00135EBE7D2
:104FC000002BA7D10B7884F8423004F1420565E745
:104FD000D65200085D53000810B50C46B1F90E100A
:104FE000FBF7F4F80028ABBF636DA3891B1823F40B
:104FF0008053ACBF6365A38110BD2DE9F0411F460E
:105000008B89DB0505460C46164605D50223002292
:10501000B1F90E10FBF7E7F8A389B4F90E1023F4E9
:105020008053A38132463B462846BDE8F041FBF75A
:10503000D1B810B50C46B1F90E10FBF7D4F8431CEB
:10504000A38915BF606523F4805343F48053A38183
:1050500018BFA38110BDB1F90E10FBF7BFB8000057
:1050600001F0FF01102A2BDB10F0070F08D010F819
:10507000013B013A8B422DD010F0070F42B3F6D11D
:10508000F0B441EA012141EA014122F007047FF036
:1050900000070023F0E80256083C85EA010586EA8D
:1050A000010685FA47F5A3FA87F586FA47F6A5FAC9
:1050B00087F68EB9EED1F0BC01F0FF0102F00702D5
:1050C00032B110F8013B013A83EA010313B1F8D180
:1050D0000020704701387047002D06BF3546033861
:1050E000073815F0010F07D1013015F4807F02BF9A
:1050F000013015F4C03F0130F0BC0138704700BFEB
:1051000070477047425553204641554C5420484102
:105110004E444C4552004445425547204D4F4E2089
:1051200048414E444C45520044554D4D592048414C
:105130004E444C45520048415244204641554C543F
:105140002048414E444C4552004D454D204D414E66
:105150004147452048414E444C4552004E4D492060
:1051600048414E444C455200555341474520464125
:10517000554C542048414E444C4552002A2A2A207E
:1051800052494F54206B65726E656C2070616E6978
:10519000633A0A25730A0A002A2A2A207265626F76
:1051A0006F74696E672E2E2E0A0A006D61696E2873
:1051B000293A20546869732069732052494F542159
:1051C000202856657273696F6E3A20323031372E5F
:1051D00030312D646576656C2D3235352D6731663D
:1051E0006232312D56616E64726973290A006964F6
:1051F0006C65006D61696E000044004000000200B3
:1052000003000240020002400700260604000000DE
:105210000048004000000400090C0240080C024055
:10522000070027030400000000000040FFFFFFFF0D
:1052300001000000001C0000000C0040FFFFFFFF09
:10524000080000000032000052494F54206E65747F
:10525000776F726B20737461636B206578616D701A
:105260006C65206170706C69636174696F6E004D6C
:105270007920616464726573732069732025730AF1
:10528000006970763600FF01000000000000000099
:10529000000000000001FE8000000000000000008F
:1052A00000000000000000000000000000000000FE
:1052B000000000000001FF020000000000000000EC
:1052C0000001FF00000000000000000000000000DE
:1052D00000000000000030313233343536373839C1
:1052E00061626364656600002C020020000000001B
:1052F00000000000000000000000000000000000AE
:10530000000000000000000000000000000000009D
:10531000000000000000000000000000000000008D
:10532000000000000000000000000000000000007D
:10533000000000000000000000000000000000006D
:10534000000000000000000000000000232D302BB2
:105350002000686C4C006566674546470030313276
:10536000333435363738394142434445460000002E
:1053700038130020000000006403002040000000FB
:105380000000000000000000EE510008F35100088A
:10539000FF000000010000002C02002000000000BF
:1053A0000C5300082C530008EC52000800000000C9
:1053B00000000000000000000000000000000000ED
:1053C00000000000000000000000000000000000DD
:1053D00000000000000000000000000000000000CD
:1053E00000000000000000000000000000000000BD
:0C53F000000000000000000000000000B1
:04000005080004717A
:00000001FF
